:020000020000FC
:0200000012C02C
:100026000FE50DBF01E00EBFDED5ECE2FFE050D6D6
:1000360030D600E000937A00959A00E000937B00AA
:100046008ED5959A8D9A959A2AD5A7D622D61C2D05
:100056001F3F09F4112719D44CD71A95E2F710E07F
:1000660014D452D3009189000030F1F426D53AD742
:1000760010D611E00AD448D3009189000030A1F4CB
:100086001CD530D706D612E000D43ED300918900A5
:10009600013051F408D51BD7FCD519D434D7F9D57E
:1000A6000091790058D6F5D5FFCF33244424552442
:1000B600089566247724882408951CD0632C742C14
:1000C600852C18D017D026D008951F931FB71F93DD
:1000D6000F9305C01F931FB71F930F930AE0602E5F
:1000E60000E0702E802E18E132D00F911F911FBFB5
:1000F6001F910895330C441C551C08951F931FB778
:10010600302E44245524E6DF032D029506291FBF11
:100116001F910895360C471C581C08953618470839
:10012600580808950F93032D362C602E042D472C66
:10013600702E032D582C802E0F9108950F931F9328
:1001460010E0300E411E511E1F910F9108959F928F
:10015600AF92BF921F932F932FB718E1212E962CA3
:10016600A72CB82C662477248824330C441C551CF1
:10017600661C771C881C69147A048B0420F06918A5
:100186007A088B0833942A9481F72FBF2F911F91F9
:10019600BF90AF909F9008956F921F931FB70F93D4
:1001A60000E1602E0F9155244424262E372E3694D6
:1001B600279410F4480E591E579447943794279461
:1001C6006A94B9F71FBF1F916F9008950F930FB7E9
:1001D600542C432C322C0FBF0F9108956F921F930E
:1001E6001FB76F937F938F939F9360917400709165
:1001F600750080917600909177000F9300E1602E54
:100206000F9155244424262E372E3694279410F425
:10021600480E591E57944794379427946A94B9F711
:100226009F918F917F916F911FBF1F916F9008953E
:100236000F931F931FB75694479437942794569459
:1002460047943794279400E8201628F001E0300EF2
:1002560000E0401E501E1FBF1F910F9108950F937F
:100266000FB70F932F9321DF222708E0169520F46E
:10027600360C471C581C30F00A9521F0660C771C8A
:10028600881CF4CF2F910F910FBF0F9108950F93F4
:100296000FB78694779467941A95D9F70FBF0F9185
:1002A60008950F930FB75694479437941A95D9F734
:1002B6000FBF0F9108950F930FB70E7F330C441C99
:1002C600551C18F01A95D1F701C001600FBF0F91A8
:1002D60008951A3340F01F7D173408F009C0113411
:1002E60038F0175303C0103318F01F708894089520
:1002F600089408950F700A300CF0095F005D0895A8
:100306002F932FB70F93F6DF102F0F910295F2DF81
:100316002FBF2F9108950F932F932227E0E6F0E049
:100326000AE0602E7724882418E111DF062D006389
:10033600019323950AE0602E772488243614470417
:10034600580494F7032D00630193239500E000837E
:10035600122F2F910F9108950F931F931FB71F937D
:100366000FEF30264026502601E010E0300E411EE9
:10037600511E1F911FBF1F910F9108950F931F9339
:100386001FB71F930FEF60267026802601E010E04E
:10039600600E711E811E1F911FBF1F910F91089540
:1003A6000F931F931FB710D00AF4D6DF1FBF1F91FC
:1003B6000F9108950F931F931FB70BD00AF4DEDF3A
:1003C6001FBF1F910F910895152D10780AF410E89C
:1003D600089510E06116710681060AF410E8089582
:1003E6000F931F93222711276F937F938F939F93CA
:1003F60060917400709175008091760090917700FD
:10040600772342F41FEF6127712711E0610F10E097
:10041600711F10E8992342F42FEF8227922721E0DB
:10042600820F20E0921F20E82127B6DE22235AF40D
:100436001FEF212631264126512611E0210E1127D4
:10044600311E411E511E9F918F917F916F911F9179
:100456000F9108951F9311272227552012F47CDF50
:1004660020E8882012F48ADF10E8212770DE222394
:100476000AF472DF1F9108954F925F926F927F92F6
:10048600712E7326112322F41095019508F0139509
:10049600332322F43095219508F033950F9300E12C
:1004A600602E0F91422E532E22273327000F111F45
:1004B600221F331F2415350518F024193509039515
:1004C6006A94A1F7772042F41095019508F01395E8
:1004D6003095219508F033957F906F905F904F90FF
:1004E6000895AF93BF930F931F932F933F933FB7F7
:1004F6003F93ADB7BEB72AE0A20F20E0B21F3D91F1
:100506001D910D9120E8212333235AF43F70000FEB
:10051600111F3A95E1F7222312F410680EC01F77D7
:100526000CC0222332F40894179507953A95D9F70B
:1005360004C0169507953A95E1F70E931E932E93F0
:100546003F913FBF3F912F911F910F91BF91AF9167
:1005560008952F933F933FB7000020E00197803026
:100566009207D1F73FBF3F912F9108952F933F9365
:100576003FB78F939F9388EE93E001C000000197E9
:1005860020E080309207D1F71A95A9F79F918F91B5
:100596003FBF3F912F9108951F9314E6E7DF1F9108
:1005A600089532B3352B32BB08951F9332B3152FFE
:1005B6001095312332BB1F91089531B3352B31BBD2
:1005C60008951F9331B3152F1095312331BB1F9119
:1005D60008951F932F932FB73F938F939F9310E008
:1005E60010937A00E2DFF894E8DF80EE91E0B1DF65
:1005F600E8DF8CE390E0ADDF10B3152321F011E0C6
:1006060010937A009598789484EA91E0A2DF9F91FE
:100616008F913F912FBF2F911F9108951F932F9375
:100626008F939F932FB7C1DFF894C7DF81E090E0E7
:1006360010E0019780309107E1F7469508F4C1DF95
:100646008CE390E086DFBDDF78949F918F912FBF7A
:100656002F911F9108954F931F932F938F939F93DD
:100666002FB740E0A2DFF894A8DF81E090E010E029
:10067600019780309107E1F7A4DF8DE090E069DF14
:1006860040B3452309F041E08FE290E062DF7894C1
:100696002FBF9F918F912F911F9146954F9108954E
:1006A6001F931FB71F937F9378E040E0D4DF4795F1
:1006B6007A95E1F77F911F911FBF1F9108951F93B0
:1006C6001FB77F9378E0AADF7A95E9F77F911FBF7E
:1006D6001F91089510918900112311F47ADF13C038
:1006E60010917B00112321F074DF4CECE8DF01C090
:1006F600E3D04EE4E4DF40E0E2DF40E0E0DF1091EB
:100706008A00412FDCDF08951F932F932FB74F9355
:1007160010917B00112321F05CDF4CECD0DF01C08F
:10072600CBD044E4CCDF97DFF0F710917B001123A8
:1007360021F04FDF4CECC3DF01C0BED04EEBBFDF74
:10074600AFDFE42EADDFF42E44DF4F912FBF2F91A4
:100756001F9108952F931F93EF92FF92DF92DFB6BA
:1007660010E11093740017E210937500EE0CFF1C55
:10077600EE0CFF1CEE0CFF1CEE0CFF1CE09276004C
:10078600F09277002DDEDFBEDF90FF90EF901F9195
:100796002F9108952F931F93EF92FF92DF92DFB66A
:1007A60010E11093740017E21093750017E0EE0C39
:1007B600FF1C1A95E1F7E0927600F092770010DEC2
:1007C600DFBEDF90FF90EF901F912F9108954F931A
:1007D600EF92FF92DF92DFB6F594E79440E04795FB
:1007E600EE0CFF1CAE2DBF2DAA0FBB1FAA0FBB1F01
:1007F600AE0DBF1D4078442331F0BB2312F0159691
:1008060002C0A550B040DF90FF90EF904F91089541
:100816004F93DF92DFB6DDDE43E351DF41DF4093E6
:100826008B003EDF40938C003BDF40938D0038DF2A
:1008360040938E0035DF40938F0032DF4093900067
:100846002FDF409391002CDF40939200DFBEDF90B4
:100856004F910895EF93FF93CF93DF932F931F93B9
:10086600E4EEFBE0E10F1127F11F1491E9E8F0E057
:100876002BE0019193D313952A95D9F71F912F91C8
:10088600DF91CF91FF91EF910895EF93FF932F930F
:100896001F93E4EEFBE0E10F1127F11F1491E9E845
:1008A600F0E02BE073D3139501932A95D9F71F91A6
:1008B6002F91FF91EF9108958CDE45E500DFEBE87F
:1008C600F0E028E04191FBDE2A95E1F708950F93C9
:1008D6004F93DF92DFB61F932F93EF93FF9300277B
:1008E6000093790010917B00112321F072DE4CEC0D
:1008F600E6DE01C0E1DF2FEF4EEBE1DEEFE7F0E0F1
:1009060019E0CEDE41932423042F0CD11A95C9F7A2
:1009160060DE2F3F21F000917900002319F021E0DD
:1009260020937A00FF91EF912F911F91DFBEDF9008
:100936004F910F910895BB24AA24992401C000C0A9
:1009460088248394982D77246624662760937900FB
:10095600992009F008C03DDE00917A000023B9F025
:1009660000E000937D0000917D00002321F00091BE
:100976008B00002339F4BB249924AA24B0927A0070
:10098600B0927D0000917D0000937E00089540EFB7
:1009960096DE772788275FDE771F5DDE881F01E0FA
:1009A600801709F006C0701721F400E000937D005F
:1009B600DACF781711F0A72F16C08B1448F4F0E0A1
:1009C600EBE8E60D0081A0E0092331F0A1E004C0C8
:1009D600A0E08B1409F4A1E0AA2329F4782C072DB2
:1009E600093008F4A72CF0E0EBE8E60D0081AA2315
:1009F60011F0092B03C0192F1095012300834A2FEC
:100A06000DDE8394990F992319F48CD0639491E0A9
:100A160008E0601620F401E4801608F4BACFB72C7B
:100A2600BB2011F49924939400917900002321F4BA
:100A360001E000937D0001C09ECF95CFCC247BDFE3
:100A460000917E00002391F012D01C2D03DF23D0ED
:100A5600992061F4C39473DF00917E00002331F086
:100A660006D01C2DF7DE17D09920A1F308951F9309
:100A76000F9310E000918B00003141F0083229F409
:100A860011E000E600938A0001C01FEF1093890071
:100A96000F911F9108950C2D18E580D2089518E541
:100AA60075D2C02E08950F9300918900002311F08E
:100AB6001BD001C002D00F9108954F93EF92FF9281
:100AC600DF92DFB6F594E79440E04795407821F051
:100AD600EE200AF4E39445E0BE2DA42FDFBEDF909E
:100AE600FF90EF904F9108954F93DF92DFB6AE2DB2
:100AF600BF2D44E0AA0FBB1F4A95E1F7BB2322F4A2
:100B0600B39540E04A1BA42F3A2E44245524D5DA47
:100B1600D4DAA42D40E8341608F0A395DFBEDF90A2
:100B26004F9108952F936F930F931F930F9318E090
:100B36006091790006270795062F10F428E1022711
:100B46000795602F0F9107950F931A9599F7609364
:100B560079000F911F910F916F912F91089554E095
:100B66008D98959A00B3007209F00895222714DD36
:100B76002395223318F500B30072C9F32431E0F44B
:100B860020917B0020937C0021E020937B0087DF6F
:100B96001C2D139528E0121750F43ADE68DF5ADE52
:100BA600C12E79DF20917C0020937B0015C0209117
:100BB6007C0020937B0012C041DF0EC02BE000E0DA
:100BC600E9E8F0E001932A95E9F717E043DE1A9584
:100BD600EAF7CC24CA945FDF8D9A9598FFCF000B75
:100BE60016212C37424D0F9303E00093780000E066
:100BF60002B90CE009B906E003B9539A549A0F9169
:100C060008951AE005E511D01A95E1F7FACF0DE23D
:100C16000CD0ECE2FFE05CD028D0E8E3FFE058D04F
:100C260038D037D008EC9BD108955D9BFECF0CB928
:100C360008950F935D9BFECF0CB90AE05D9BFECF36
:100C46000CB90DE05D9BFECF0CB90F9108955F9B2B
:100C5600FECF0CB108955F9BFECF0CB11F93109190
:100C6600780010FDE2DF1F9108950F9300E2DDDFAB
:100C76000F9108950F930AE2D8DF0F9108950F930D
:100C86000AE0D3DF0F9108950F930DE0CEDF0F91A9
:100C960008950F931F931FB70AE0C7DF0DE0C5DF66
:100CA6001FBF1F910F9108950F9304E0BEDF0F91B0
:100CB60008950F930BE3B9DF0F9108950F930CE29C
:100CC600B4DF0F9108950F9309E0AFDF0F910895F8
:100CD6000F93EF93FF930FB70F930591003011F029
:100CE600A4DFFBCF0F910FBFFF91EF910F910895F6
:100CF60054D000E29ACF51D0CCCFEF93FF93E0E2ED
:100D0600FFE0E6DFC6DFFF91EF910895EF93FF93D3
:100D1600E6E2FFE0DDDFBDDFFF91EF9108951F936F
:100D26002F9399DF102FD5DAE0F3212F229593DF49
:100D3600102FCFDAE0F3012F022B2F911F91089588
:100D46008ADF0F70000F102E110C110C100E83DFAE
:100D56000F70010D08950F931F93D2DA66DF012FEE
:100D660064DF1F910F9108950F931F932F932FB751
:100D76002F93EF93FF9328E0102F110F10F000E34D
:100D860001C001E352DF2A95C1F7FF91EF912F9140
:100D96002FBF2F911F910F9108950F931F932F939C
:100DA6002FB7102F00E36894145610F00395FCCF6C
:100DB600003311F03ADFE8941C5900E31A5010F0A2
:100DC6000395FCCF16F4003309F02FDF165F00E31E
:100DD600010F2BDF2FBF2F911F910F9108953F9386
:100DE6003FB73F924F925F925524302E412E25D029
:100DF6005F904F903F903FBF3F9108950F931F9391
:100E06001FB7E0E6F0E0222426DF0FDF0D3021F0E9
:100E16000F7001932394F8CF5F9919DF332444248C
:100E26005524E0E6F0E0019189D92A9411F045D9DC
:100E3600FACF1FBF1F910F9108950F931F93EF9342
:100E4600FF9369DA0291F1DE1A95E1F7FF91EF91CE
:100E56001F910F9108950F930FB70F93B5DA1AF4F8
:100E66007BDA0DE2E2DEE9DF0F910FBF0F91089505
:100E76001F931FB72F93202F222322F421950DE2D3
:100E8600D4DE022F8ADF2F911FBF1F9108953F9353
:100E96003FB73F924F925F92552411230AF45A941A
:100EA600302E412ED8DF5F904F903F903FBF3F914D
:100EB60008950F931F931FB700918900002311F027
:100EC60006D001C00FD01FBF1F910F9108950B2FA1
:100ED600CFDF0CE2AADEAA3010F400E3A6DE0A2F6A
:100EE6005CDF08950B2FC4DF0CE29FDE0A2F55DF6F
:100EF6000895E9E8F0E02AE001912DDFB6DE2A95B3
:100F0600D9F7C7DE0895EFE7F0E029E0019123DF86
:100F1600B1DE2A95D9F7BDDE0895444F4E4500004F
:100F26004552524F520048616C6C6F2057656C7485
:100F3600000052455620302E31000F930FB70F9305
:100F460000E5000000000A95E1F70F910FBF0F9131
:100F560008950F930FB70F931F9302E40DC01F93CD
:100F66001FB7F7DF0A95E9F71FBF1F9108950F9383
:100F76000FB70F931F9306E119EC1A95F1F70A952F
:100F8600D9F71F910F910FBF0F910895E199FECFE9
:100F9600F8941EBBE09A0DB378940895E199FECFBC
:0E0FA600F8941EBB0DBBE29AE19A7894089570
:00000001FF
